:020000040000FA
:06000000CA3001303A286D
:08000800A000030EA100831209
:1000100005191028831601178312B23081002B288E
:1000200083160113831203140B190310A80DA90DD5
:10003000AA0DAB0DAC0DAC16FF302C02031D2B2806
:10004000FA302B02031D2B2831152A08AF0029088E
:10005000AE002808AD008B100B11210E8300A00EFE
:04006000200E090065
:0C007400203084008001840A80300402E7
:10008000031C3C281230B000E02183160C3085059B
:1000900087018312850187010730990000309A009B
:1000A000103083168E008312603083168F00831207
:1000B0000030831691009F008312C83083168100A0
:1000C000831231309000003083168C008312103080
:1000D0008B00831600309B001C141A088312BC008E
:1000E000851DD822831610309B001C141A08831219
:1000F000BD00831630309B001C141A088312DE00EA
:10010000BF2281018E018F010B118B100B108C010E
:100110008B17982031199B20B30B96280310851953
:100120000314B90DF0303902031944211E23892824
:1001300064003210080031110130B7008B132030F9
:10014000370783169B001C141A088312A400103072
:10015000370783169B001C141A088312A300A600FD
:100160000230A6060030370783169B001C141A08BD
:100170008312A200A7000130A7068B17321CC628E5
:1001800022090339A200A309A409A50924082F0202
:10019000031D3E2923082E02031D3E2922082D029D
:1001A000031D3E2901303702031DDB283D18DB28E3
:1001B0003D143E14ED2102303702031DE428BD1822
:1001C000E428BD143E14FC2103303702031DED2842
:1001D0003D19ED283D153E14082204303702031D59
:1001E000F628BD19F628BD153E1414220530370235
:1001F000031DFF283D1AFF283D163E14232206301A
:100200003702031D0829BD1A0829BD163E143222E3
:1002100007303702031D11293D1B11293D173E14DC
:10022000412208303702031D1A29BD1B1A29BD17A8
:100230003E144C2209303702031D23295E1823295E
:100240005E143E1457220A303702031D2C29DE1893
:100250002C29DE143E1462220B303702031D35298F
:100260005E1935295E153E146D220C303702031DD0
:100270003E29DE193E29DE153E147822B70A0D30DC
:100280003702031808009E280130B600B300B400FE
:10029000B500B70085018701B1139820B30B8C29F5
:1002A000031085190314B90DF03039020319B3296D
:1002B000B40B8C2901303702031983220230370234
:1002C000031988220330370203198D2204303702C4
:1002D000031992220530370203199722063037029C
:1002E00003199C22073037020319A1220830370274
:1002F0000319A622093037020319AB220A3037024C
:100300000319B0220B3037020319B5220C30370223
:100310000319BA229630B400311D4D293111321C17
:1003200096292D090339AD00AE09AF092F1C4D29BF
:100330008E018F010C1C4D290C102E1E4D298B1384
:1003400020303707BB002F08BA00CB211030370709
:10035000BB002E08BA00CB2100303707BB002D08A8
:10036000BA00CB218B1785018701B70AB6010D3082
:100370003702031C4D29BF2208003E1C08003E1016
:100380001030BB003D08BA00CB213030BB005E0806
:10039000BA00CB2108008B133A0883161C159A006B
:1003A00083123B0883169B0055309D00AA309D00A8
:1003B0009C1464009C18D9291C1183128B17080007
:1003C000FF30C800CA15CB15CC15CD15CE15CF15ED
:1003D000D015D115D215D3150800C130BD05FF3099
:1003E000DE051130C405C0000030C200C600BC18D4
:1003F0005F14BC18DF140800C230BD05FF30DE05F5
:100400000230C405C0000030C200C6005F10080002
:10041000C430BD05FF30DE050630C405C000003025
:10042000C200C6005F100800C830BD05FF30DE0501
:100430001830C405C0000030C200C600BC185F14EC
:10044000BC18DF140800D030BD05FF30DE053030A9
:10045000C405C0000030C200C600BC185F14BC1840
:10046000DF140800E030BD05FF30DE053030C40584
:10047000C0002030C200C600BC185F14BC18DF14D6
:1004800008007F30BD05C030DE05C030C505C100A5
:100490000030C300C7000800BF30BD05C030DE0516
:1004A0003030C505C1000030C300C70008003F3030
:1004B000BD05C130DE059030C505C1000030C30068
:1004C000C70008003F30BD05C230DE05C030C5059D
:1004D000C1000030C300C70008003F30BD05C43074
:1004E000DE05C030C505C1000030C300C7000800EC
:1004F0003F30BD05C830DE05C030C505C100003045
:10050000C300C700080010308506023087060800C7
:10051000203085060030870608002130850600302F
:100520008706080002308506023087060800003082
:1005300085060630870608000030850606308706E7
:10054000080000308706183087060800003085064E
:10055000213087060800003085060930870608002C
:1005600000308706183087060800003087061830EC
:1005700087060800003087061830870608003D18F7
:10058000ED21BD18FC213D190822BD1914223D1A88
:100590002322BD1A32223D1B4122BD1B4C225E1874
:1005A0005722DE1862225E196D22DE1978220800B9
:1005B000B601B301B4013C1CE02ABC01BC14E22A20
:1005C000BC013C143C08B6006400E62AE72AE82A8D
:1005D000E92AEA2AFF30B41B8500B41F8501B30B5A
:1005E000E42AB40BE42A0310B60CB608031DE42A6F
:1005F0000030BB003C08BA00CB21080005125C1893
:100600000516DC1C8512DC1885165C1D05105C19AE
:100610000514DC1D8510DC1985145C1E87105C1A1E
:100620008714DC1E0711DC1A07155C1F07105C1B02
:100630000714DC1F8712DC1B871608008F080319BC
:1006400008008F0178308E00C80F502DC80A441C56
:100650004E2B461C3F2BCA1C302BCA014A155C2B63
:100660004A1D352BCA01CA155C2BCA1D3A2BCA017B
:100670004A165C2B4A1E5C2BCA01CA145C2B4A1D0D
:10068000442BCA014A165C2BCA1D492BCA014A16C3
:100690005C2B4A1E5C2BCA01CA145C2BCA1C532B50
:1006A000CA014A155C2B4A1D582BCA01CA155C2B7E
:1006B0004A1E5C2BCA014A15C41C832BC61C742B12
:1006C000CB1C652BCB014B15912B4B1D6A2BCB0102
:1006D000CB15912BCB1D6F2BCB014B16912B4B1EAA
:1006E000912BCB01CB14912B4B1D792BCB014B16AE
:1006F000912BCB1D7E2BCB014B16912B4B1E912B9F
:10070000CB01CB14912BCB1C882BCB014B15912B00
:100710004B1D8D2BCB01CB15912B4B1E912BCB0160
:100720004B15441DB82B461DA92BCC1C9A2BCC0174
:100730004C15C62B4C1D9F2BCC01CC15C62BCC1DAC
:10074000A42BCC014C16C62B4C1EC62BCC01CC14B2
:10075000C62B4C1DAE2BCC014C16C62BCC1DB32B7F
:10076000CC014C16C62B4C1EC62BCC01CC14C62B70
:10077000CC1CBD2BCC014C15C62B4C1DC22BCC0167
:10078000CC15C62B4C1EC62BCC014C15C41DEE2B14
:10079000C61DDF2BCD1CD02BCD014D155F13FC2BBF
:1007A0004D1DD52BCD01CD15FC2BCD1DDA2BCD014B
:1007B0004D16FC2B4D1EFC2BCD01CD14FC2B4D1DDD
:1007C000E42BCD014D16FC2BCD1DE92BCD014D1693
:1007D000FC2B4D1EFC2BCD01CD14FC2BCD1CF32B83
:1007E000CD014D15FC2B4D1DF82BCD01CD15FC2B4E
:1007F0004D1EFC2BCD014D155F1B252C441E252CB9
:10080000461E162CCE1C072CCE014E15332C4E1D29
:100810000C2CCE01CE15332CCE1D112CCE014E1634
:10082000332C4E1E332CCE01CE14332C4E1D1B2CDC
:10083000CE014E16332CCE1D202CCE014E16332C5D
:100840004E1E332CCE01CE14332CCE1C2A2CCE01BE
:100850004E15332C4E1D2F2CCE01CE15332C4E1E93
:10086000332CCE014E15C41E5A2CC61E4B2CCF1C49
:100870003C2CCF014F15682C4F1D412CCF01CF15BB
:10088000682CCF1D462CCF014F16682C4F1E682CAC
:10089000CF01CF14682C4F1D502CCF014F16682C60
:1008A000CF1D552CCF014F16682C4F1E682CCF0141
:1008B000CF14682CCF1C5F2CCF014F15682C4F1D17
:1008C000642CCF01CF15682C4F1E682CCF014F151B
:1008D000DF18912C451E912C471E822CD01C732CA6
:1008E000D00150159F2C501D782CD001D0159F2C75
:1008F000D01D7D2CD00150169F2C501E9F2CD00156
:10090000D0149F2C501D872CD00150169F2CD01D29
:100910008C2CD00150169F2C501E9F2CD001D0142F
:100920009F2CD01C962CD00150159F2C501D9B2C19
:10093000D001D0159F2C501E9F2CD0015015DF18D0
:10094000C82CC51EC82CC71EB92CD11CAA2CD1017D
:100950005115D62C511DAF2CD101D115D62CD11D3E
:10096000B42CD1015116D62C511ED62CD101D11444
:10097000D62C511DBE2CD1015116D62CD11DC32C05
:10098000D1015116D62C511ED62CD101D114D62C02
:10099000D11CCD2CD1015115D62C511DD22CD101F9
:1009A000D115D62C511ED62CD1015115DF18002D92
:1009B000451F002D471FF12CD21CE22CD2015215ED
:1009C000DF130E2D521DE72CD201D2150E2DD21D94
:1009D000EC2CD20152160E2D521E0E2DD201D21425
:1009E0000E2D521DF62CD20152160E2DD21DFB2CAF
:1009F000D20152160E2D521E0E2DD201D2140E2DE2
:100A0000D21C052DD20152150E2D521D0A2DD201D8
:100A1000D2150E2D521E0E2DD2015215DF18392D72
:100A2000DF1B392DC51F392DC71F2A2DD31C1B2DA8
:100A3000D3015315472D531D202DD301D315472D19
:100A4000D31D252DD3015316472D531E472DD301FA
:100A5000D314472D531D2F2DD3015316472DD31DCE
:100A6000342DD3015316472D531E472DD301D314D4
:100A7000472DD31C3E2DD3015315472D531D432D18
:100A8000D301D315472D531E472DD3015315BD2137
:100A90004008C4004108C5005F18DF145F1CDF1068
:100AA0004808C9000C304A05031D05120C304B05DF
:100AB000031D85120C304C05031D05100C304D052F
:100AC000031D85100C304E05031D87100C304F059B
:100AD000031D07110C305005031D07100C30510584
:100AE000031D87120C305205031D07120C305305ED
:100AF000031D871149080E020318AA2D12304A055A
:100B0000031D051612304B05031D851612304C05CA
:100B1000031D051412304D05031D851412304E05BA
:100B2000031D871412304F05031D071512305005A1
:100B3000031D071412305105031D8716123052058C
:100B4000031D071612305305031D8715FF30480299
:100B5000031908008F08031D0800982049080E0299
:100B6000031CAA2D18304A05031D051206304A053C
:100B7000031D051618304B05031D851206304B0565
:100B8000031D851618304C05031D051006304C0555
:100B9000031D051418304D05031D851006304D0545
:100BA000031D851418304E05031D871006304E05B1
:100BB000031D871418304F05031D071106304F051C
:100BC000031D071518305005031D0710063050058A
:100BD000031D071418305105031D871206305105F7
:100BE000031D871618305205031D071206305205E3
:100BF000031D071618305305031D871106305305D2
:060C0000031D871508002A
:084000000200030004000100AE
:02400E00CC33B1
:10420000010078007A007C007E007B0079007F004E
:104210007D007A0078007E007C007D007F00FF003A
:104220000200F200F600FA00FE00F200F600FA00CA
:10423000FE00F200F600FA00FE00F200F600FF00B9
:10424000FF00050005000500050009000900090040
:1042500009000D000D000D000D0011001100FF0000
:104260000100FF00FF00FF00FF00FF00FF00FF0054
:10427000FF00FF00FF00FF00FF00FF00FF00FF0046
:10428000FF00FF00FF00FF00FF00FF00FF00FF0036
:10429000FF00FF00FF00FF00FF00FF00FF00FF0026
:1042A000FF00FF00FF00FF00FF00FF00FF00FF0016
:1042B000FF00FF00FF00FF00FF00FF00FF00FF0006
:1042C000FF00FF00FF00FF00FF00FF00FF00FF00F6
:1042D000FF00FF00FF00FF00FF00FF00FF00FF00E6
:1042E000FF00FF00FF00FF00FF00FF00FF00FF00D6
:1042F000FF00FF00FF00FF00FF00FF00FF00DD00E8
:00000001FF
